:1000000072C000009EC000009CC000009AC00000AA
:1000100098C0000096C0000094C0000092C000008C
:1000200090C000004AC3000048C3000046C300005F
:1000300088C0000086C0000084C0000082C00000AC
:1000400080C000007EC000007CC000007AC00000BC
:1000500078C0000076C0000074C00000E4C2000058
:1000600070C00000AAC200007FC200006AC0000089
:1000700068C0000066C0000064C0000062C00000EC
:1000800060C000005EC000005CC000005AC00000FC
:1000900058C0000056C0000054C0000052C000000C
:1000A00050C000004EC000004CC000004AC000001C
:1000B00048C0000046C0000044C0000042C000002C
:1000C00040C000003EC000003CC000003AC000003C
:1000D00038C0000036C0000011C20000E6C10000B8
:1000E00030C00000670311241FBECFEFD1E2DEBF96
:1000F000CDBF00E00CBF12E0A0E0B2E0E0EBF8E022
:1001000000E00BBF02C007900D92A231B107D9F7F2
:1001100023E0A2E1B2E001C01D92A735B207E1F7EA
:1001200010E0C3E7D0E000E005C021970109802F6F
:10013000FE01B4D3C237D10780E00807B1F71AD364
:10014000B5C35ECFFC01A089B18982E08C93A48500
:10015000B5851C92A685B7858FEC8C93108EA489EB
:10016000B58986E08C93A289B3898C9180618C9348
:10017000A289B3898C9188608C93A289B3898C9170
:1001800080688C930288F389E02D80818F7D808345
:100190000895AF92BF92CF92DF92EF92FF920F93AA
:1001A0001F93CF93DF936C017B018B01040F151F0D
:1001B000EB015E01AE18BF08C017D10759F0699175
:1001C000D601ED91FC910190F081E02DC6011995C9
:1001D000892B79F7C501DF91CF911F910F91FF9086
:1001E000EF90DF90CF90BF90AF900895FC01538DBA
:1001F000448D252F30E0842F90E0821B930B541701
:1002000010F0CF96089501970895FC01918D828D8D
:10021000981761F0A28DAE0FBF2FB11D5D968C9126
:10022000928D9F5F9F73928F90E008958FEF9FEF65
:100230000895FC01918D828D981731F0828DE80F21
:10024000F11D858D90E008958FEF9FEF0895FC01DB
:10025000918D228D892F90E0805C9F4F821B9109A8
:100260008F73992708958DE192E0F1DF21E0892BCA
:1002700009F420E0822F08958AEB92E0E8DF21E084
:10028000892B09F420E0822F0895FC01A48DA80F8A
:10029000B92FB11DA35ABF4F2C91848D90E00196C8
:1002A0008F739927848FA689B7892C93A089B189E8
:1002B0008C91837080648C93938D848D981306C089
:1002C0000288F389E02D80818F7D80830895EF92ED
:1002D000FF920F931F93CF93DF93EC0181E0888F00
:1002E0009B8D8C8D98131AC0E889F989808185FFD0
:1002F00015C09FB7F894EE89FF896083E889F98972
:1003000080818370806480839FBF81E090E0DF9173
:10031000CF911F910F91FF90EF900895F62E0B8DC6
:1003200010E00F5F1F4F0F731127E02E8C8D8E1181
:100330000BC00FB607FCFACFE889F989808185FFE9
:10034000F5CFCE01A2DFF2CFEB8DEC0FFD2FF11D2B
:10035000E35AFF4FF0829FB7F8940B8FEA89FB892D
:1003600080818062D0CFCF93DF93EC01888D88238A
:10037000B1F0AA89BB89E889F9898C9185FD03C010
:10038000808186FD0CC00FB607FCF7CF8C9185FFEE
:10039000F2CF808185FFEDCFCE0177DFEACFDF910D
:1003A000CF91089580E090E0892B21F065DF8111E5
:1003B0000E94000080E090E0892B49F080E090E00E
:1003C000892B29F00E94000081110E94000080E02A
:1003D00090E0892B49F080E090E0892B29F00E9481
:1003E000000081110E94000080E090E0892B21F044
:1003F0003ADF81110C94000008953FB7F894809182
:10040000190290911A02A0911B02B0911C0226B50C
:10041000A89B05C02F3F19F00196A11DB11D3FBF3C
:10042000BA2FA92F982F8827BC01CD01620F711D0B
:10043000811D911D42E0660F771F881F991F4A9505
:10044000D1F708958F929F92AF92BF92CF92DF9291
:10045000EF92FF92D2DF4B015C0182E3C82ED12CD8
:10046000E12CF12CCADF681979098A099B09683ED9
:10047000734081059105B0F321E0C21AD108E1086B
:10048000F10888EE880E83E0981EA11CB11CC114EF
:10049000D104E104F10431F7FF90EF90DF90CF90A9
:1004A000BF90AF909F908F9008951F920F920FB6BC
:1004B0000F9211240BB60F922F933F934F935F939C
:1004C0006F937F938F939F93AF93BF93EF93FF931C
:1004D0008DE192E0DADEFF91EF91BF91AF919F91B4
:1004E0008F917F916F915F914F913F912F910F90DD
:1004F0000BBE0F900FBE0F901F9018951F920F927A
:100500000FB60F9211240BB60F922F938F939F93D8
:10051000EF93FF93E0912D02F0912E028081E09104
:100520003302F091340282FD1DC090818091360229
:100530008F5F8F7320913702821741F0E09136026E
:10054000F0E0E35EFD4F958F80933602FF91EF91CF
:100550009F918F912F910F900BBE0F900FBE0F9018
:100560001F9018958081F2CF1F920F920FB60F92B5
:1005700011240BB60F922F933F934F935F936F937A
:100580007F938F939F93AF93BF93EF93FF938AEBE8
:1005900092E07BDEFF91EF91BF91AF919F918F91A0
:1005A0007F916F915F914F913F912F910F900BBE73
:1005B0000F900FBE0F901F9018951F920F920FB6BD
:1005C0000F9211240BB60F922F938F939F93EF935B
:1005D000FF93E091CA02F091CB028081E091D002BA
:1005E000F091D10282FD1DC090818091D3028F5F76
:1005F0008F732091D402821741F0E091D302F0E092
:10060000E654FD4F958F8093D302FF91EF919F9118
:100610008F912F910F900BBE0F900FBE0F901F90D8
:1006200018958081F2CF1F920F920FB60F9211246E
:100630002F933F938F939F93AF93BF938091150216
:1006400090911602A0911702B091180230911402F5
:1006500023E0230F2D3758F50196A11DB11D2093DE
:1006600014028093150290931602A0931702B09380
:1006700018028091190290911A02A0911B02B09168
:100680001C020196A11DB11D8093190290931A02BC
:10069000A0931B02B0931C02BF91AF919F918F91C9
:1006A0003F912F910F900FBE0F901F90189526E845
:1006B000230F0296A11DB11DD2CF1F920F920FB62C
:1006C0000F9211240F900FBE0F901F901895EDE11F
:1006D000F2E01382128248EE53E060E070E044835F
:1006E00055836683778384E092E09183808325E35A
:1006F00031E03587248724E331E03787268720E3FC
:1007000031E0318B208B21E331E0338B228B22E3EC
:1007100031E0358B248B26E331E0378B268B118E2D
:10072000128E138E148EEAEBF2E01382128244834F
:100730005583668377839183808385EC90E09587EA
:10074000848784EC90E09787868780EC90E0918B9B
:10075000808B81EC90E0938B828B82EC90E0958B88
:10076000848B86EC90E0978B868B118E128E138E85
:10077000148E0895789484B5826084BD84B58160B8
:1007800084BD85B5826085BD85B5816085BD80915C
:100790006E00816080936E001092810080918100D4
:1007A00082608093810080918100816080938100CC
:1007B000809180008160809380008091B10084608E
:1007C0008093B1008091B00081608093B0008091EF
:1007D000910082608093910080919100816080936C
:1007E0009100809190008160809390008091A100A1
:1007F00082608093A1008091A10081608093A1001C
:100800008091A00081608093A0008091210182608E
:100810008093210180912101816080932101809149
:10082000200181608093200180917A008460809310
:100830007A0080917A00826080937A0080917A00B9
:10084000816080937A0080917A00806880937A003A
:100850001092C1008AEB92E075DC8DE192E072DCCF
:100860008DE192E0F4DC892B49F08DE192E0CDDC62
:10087000682F8AEB92E02BDDE5DDF2CF8AEB92E088
:10088000E6DC892B49F08AEB92E0BFDC682F8DE132
:1008900092E01DDDD7DDF2CF85DDE2CFEE0FFF1F49
:1008A000881F8BBF0790F691E02D1994F894FFCF25
:1008B000000000006701C900F600B301270105012F
:0208C00019011C
:00000001FF
